BL51 BANKED LINKER/LOCATER V6.22.2.0                                                    04/07/2022  22:01:02  PAGE 1


BL51 BANKED LINKER/LOCATER V6.22.2.0, INVOKED BY:
C:\KEIL_V5\C51\BIN\BL51.EXE .\Objects\main.obj, .\Objects\delay.obj TO .\Objects\MCU_1 PRINT (.\Listings\MCU_1.m51)


MEMORY MODEL: LARGE


INPUT MODULES INCLUDED:
  .\Objects\main.obj (MAIN)
  .\Objects\delay.obj (DELAY)
  C:\KEIL_V5\C51\LIB\C51L.LIB (?C_STARTUP)
  C:\KEIL_V5\C51\LIB\C51L.LIB (?C?UIDIV)
  C:\KEIL_V5\C51\LIB\C51L.LIB (?C?ULCMP)
  C:\KEIL_V5\C51\LIB\C51L.LIB (?C?LSTXDATA)
  C:\KEIL_V5\C51\LIB\C51L.LIB (?C?LSTKXDATA)
  C:\KEIL_V5\C51\LIB\C51L.LIB (?C_INIT)


LINK MAP OF MODULE:  .\Objects\MCU_1 (MAIN)


            TYPE    BASE      LENGTH    RELOCATION   SEGMENT NAME
            -----------------------------------------------------

            * * * * * * *   D A T A   M E M O R Y   * * * * * * *
            REG     0000H     0008H     ABSOLUTE     "REG BANK 0"
            IDATA   0008H     0001H     UNIT         ?STACK

            * * * * * * *  X D A T A   M E M O R Y  * * * * * * *
            XDATA   0000H     001EH     UNIT         ?XD?MAIN

            * * * * * * *   C O D E   M E M O R Y   * * * * * * *
            CODE    0000H     0003H     ABSOLUTE     
                    0003H     0008H                  *** GAP ***
            CODE    000BH     0003H     ABSOLUTE     
            CODE    000EH     00C1H     UNIT         ?PR?MAIN?MAIN
            CODE    00CFH     00B1H     UNIT         ?PR?NUM_DISPLAY?MAIN
            CODE    0180H     00A3H     UNIT         ?C?LIB_CODE
            CODE    0223H     008CH     UNIT         ?C_C51STARTUP
            CODE    02AFH     0087H     UNIT         ?PR?TIME?MAIN
            CODE    0336H     0029H     UNIT         ?PR?SETCONFIG?MAIN
            CODE    035FH     0015H     UNIT         ?C_INITSEG
            CODE    0374H     000EH     UNIT         ?PR?_DELAY?DELAY



OVERLAY MAP OF MODULE:   .\Objects\MCU_1 (MAIN)


SEGMENT
  +--> CALLED SEGMENT
---------------------
?C_C51STARTUP
  +--> ?PR?MAIN?MAIN
  +--> ?C_INITSEG

?PR?MAIN?MAIN
  +--> ?PR?SETCONFIG?MAIN
BL51 BANKED LINKER/LOCATER V6.22.2.0                                                  04/07/2022  22:01:02  PAGE 2


  +--> ?PR?NUM_DISPLAY?MAIN

?PR?NUM_DISPLAY?MAIN
  +--> ?PR?_DELAY?DELAY



SYMBOL TABLE OF MODULE:  .\Objects\MCU_1 (MAIN)

  VALUE           TYPE          NAME
  ----------------------------------

  -------         MODULE        MAIN
  C:0000H         SYMBOL        _ICE_DUMMY_
  D:0080H         PUBLIC        P0
  D:0090H         PUBLIC        P1
  D:00A0H         PUBLIC        P2
  D:00B0H         PUBLIC        P3
  B:00A8H.7       PUBLIC        EA
  D:00A8H         PUBLIC        IE
  D:00B8H         PUBLIC        IP
  X:0000H         PUBLIC        TH
  X:0002H         PUBLIC        TL
  C:000EH         PUBLIC        main
  C:0336H         PUBLIC        setConfig
  X:0004H         PUBLIC        count
  C:00CFH         PUBLIC        num_display
  C:02AFH         PUBLIC        time
  D:0098H         PUBLIC        SCON
  D:0089H         PUBLIC        TMOD
  D:0088H         PUBLIC        TCON
  X:0008H         PUBLIC        bd
  B:00A8H.1       PUBLIC        ET0
  X:000AH         PUBLIC        ge
  D:008CH         PUBLIC        TH0
  D:008DH         PUBLIC        TH1
  D:008AH         PUBLIC        TL0
  X:000CH         PUBLIC        num
  D:008BH         PUBLIC        TL1
  B:0088H.4       PUBLIC        TR0
  B:0088H.6       PUBLIC        TR1
  X:000EH         PUBLIC        qm
  X:0010H         PUBLIC        ui
  X:0012H         PUBLIC        wj
  D:00C8H         PUBLIC        T2CON
  D:00D0H         PUBLIC        PSW
  X:0014H         PUBLIC        num_var
  -------         PROC          SETCONFIG
  C:0336H         LINE#         9
  C:0336H         LINE#         10
  C:0336H         LINE#         11
  C:033FH         LINE#         12
  C:0346H         LINE#         15
  C:0349H         LINE#         16
  C:034CH         LINE#         17
  C:034FH         LINE#         18
  C:0352H         LINE#         19
BL51 BANKED LINKER/LOCATER V6.22.2.0                                                  04/07/2022  22:01:02  PAGE 3


  C:0354H         LINE#         20
  C:0356H         LINE#         21
  C:0358H         LINE#         24
  C:035AH         LINE#         25
  C:035CH         LINE#         28
  C:035EH         LINE#         29
  -------         ENDPROC       SETCONFIG
  -------         PROC          NUM_DISPLAY
  C:00CFH         LINE#         9
  C:00CFH         LINE#         10
  C:00CFH         LINE#         11
  C:00D2H         LINE#         12
  C:00E5H         LINE#         13
  C:00ECH         LINE#         14
  C:00EFH         LINE#         16
  C:00F2H         LINE#         17
  C:0105H         LINE#         18
  C:010CH         LINE#         19
  C:010FH         LINE#         21
  C:0112H         LINE#         22
  C:0125H         LINE#         23
  C:012CH         LINE#         24
  C:012FH         LINE#         26
  C:0132H         LINE#         27
  C:0145H         LINE#         28
  C:014CH         LINE#         29
  C:014FH         LINE#         31
  C:0152H         LINE#         32
  C:0165H         LINE#         33
  C:016CH         LINE#         34
  C:016FH         LINE#         36
  C:0172H         LINE#         37
  C:0175H         LINE#         38
  C:017CH         LINE#         39
  C:017FH         LINE#         40
  -------         ENDPROC       NUM_DISPLAY
  -------         PROC          TIME
  C:02AFH         LINE#         43
  C:02CCH         LINE#         46
  C:02CFH         LINE#         47
  C:02D2H         LINE#         48
  C:02ECH         LINE#         49
  C:02ECH         LINE#         50
  C:02EEH         LINE#         51
  C:02F0H         LINE#         52
  C:02FCH         LINE#         54
  C:02FCH         LINE#         59
  C:031BH         LINE#         60
  -------         ENDPROC       TIME
  -------         PROC          MAIN
  C:000EH         LINE#         63
  C:000EH         LINE#         64
  C:000EH         LINE#         66
  C:0011H         LINE#         67
  C:0011H         LINE#         68
  C:0011H         LINE#         69
  C:0017H         LINE#         70
BL51 BANKED LINKER/LOCATER V6.22.2.0                                                  04/07/2022  22:01:02  PAGE 4


  C:0017H         LINE#         71
  C:002BH         LINE#         73
  C:0045H         LINE#         74
  C:0065H         LINE#         75
  C:0089H         LINE#         76
  C:00A9H         LINE#         77
  C:00C0H         LINE#         79
  C:00C3H         LINE#         80
  C:00C5H         LINE#         81
  C:00C7H         LINE#         82
  C:00C9H         LINE#         83
  C:00C9H         LINE#         84
  C:00CCH         LINE#         85
  -------         ENDPROC       MAIN
  -------         ENDMOD        MAIN

  -------         MODULE        DELAY
  C:0000H         SYMBOL        _ICE_DUMMY_
  C:0374H         PUBLIC        _delay
  -------         PROC          _DELAY
  D:0006H         SYMBOL        i
  C:0374H         LINE#         3
  C:0374H         LINE#         5
  C:0374H         LINE#         6
  C:0381H         LINE#         7
  -------         ENDPROC       _DELAY
  -------         ENDMOD        DELAY

  -------         MODULE        ?C?UIDIV
  C:0180H         PUBLIC        ?C?UIDIV
  -------         ENDMOD        ?C?UIDIV

  -------         MODULE        ?C?ULCMP
  C:01D5H         PUBLIC        ?C?ULCMP
  -------         ENDMOD        ?C?ULCMP

  -------         MODULE        ?C?LSTXDATA
  C:01E6H         PUBLIC        ?C?LSTXDATA
  -------         ENDMOD        ?C?LSTXDATA

  -------         MODULE        ?C?LSTKXDATA
  C:01F2H         PUBLIC        ?C?LSTKXDATA
  -------         ENDMOD        ?C?LSTKXDATA

Program Size: data=9.0 xdata=30 code=890
LINK/LOCATE RUN COMPLETE.  0 WARNING(S),  0 ERROR(S)
